:020000040800F2
:10000000A804002005010008290100082B010008B0
:100010002D0100082F010008310100080000000038
:100020000000000000000000000000003301000894
:100030003501000800000000370100083901000800
:100040003B0100083B0100083B0100083B010008A0
:100050003B0100083B0100083B0100083B01000890
:100060003B0100083B0100083B0100083B01000880
:100070003B0100083B0100083B0100083B01000870
:100080003B0100083B0100083B0100083B01000860
:100090003B0100083B0100083B0100083B01000850
:1000A0003B010008ED0500083B010008E1040008E1
:1000B0000506000815070008410800083B01000874
:1000C0003B0100083B0100083B0100083B01000820
:1000D0003B0100083B0100083B0100083B01000810
:1000E0003B0100083B0100083B010008DFF810D08D
:1000F00000F02EF800480047090A0008AFF300801E
:10010000A80400200D488047DFF83400016841F45E
:10011000E0210160BFF34F8FDFF82800DFF82810DF
:1001200001600A4800477047FEE7FEE7FEE7FEE78A
:10013000FEE7FEE7FEE7FEE7FEE7FEE72701000831
:1001400024ED00E00CED00E00003FA05ED000008EE
:10015000064C074D06E0E06840F0010394E8070014
:1001600098471034AC42F6D3FFF7C4FF700A00087A
:10017000900A00082DE9F041DFF8C4C0314B60451A
:1001800003D19C6944F400649C614FF08046B04206
:1001900003D1DC6944F00104DC612B4DA84203D19A
:1001A000DC6944F00204DC61284FB84203D1DC6909
:1001B00044F00404DC61838943F0010383810F2947
:1001C00000D90F21224C4FF0E02360450CD1226171
:1001D000DFF880804FEA011C88F800C0D3F800C126
:1001E0004CF0007CC3F800C1B0420DD16261DFF871
:1001F00064C00E010CF1030C8CF80060D3F80061B0
:1002000046F08056C3F80061A8420AD1A261114E9F
:100210000D01361D3570D3F8005145F00055C3F877
:100220000051B8420AD1E26108010A49491D08702B
:10023000D3F8000140F08040C3F80001BDE8F08130
:10024000002C014000100240000400400008004063
:100250000000002019E400E070B5194C83202060F4
:1002600000256560A56017486060012000F044F833
:1002700061680843606014490D60086840F002003E
:100280000860206840F48030206020688003FCD53E
:10029000206840F08070206020688001FCD5606894
:1002A00020F003006060606840F0020060606068F9
:1002B00040F480006060086840F01000086070BD85
:1002C0000010024000841D000020024000487047DA
:1002D00000A24A040549064A884202D005498842DC
:1002E00001D110467047104670470000002C0140B5
:1002F00000A24A0400340140012804D0B0F5807FF8
:1003000003DD012102E000202CE00021802801DD36
:10031000012200E000220A44402801DD012100E022
:1003200000210A44102801DD012100E000210A44D7
:10033000082801DD012100E000210A44042801DD34
:10034000012100E000210A44022801DD012100E032
:1003500000211144012801DD012000E000200844B3
:10036000C01D0001702800D100207047012181408C
:1003700001480160704700001408014001218140DC
:1003800001480160704700001008014001218140D0
:100390000148016070470000140C014001218140B8
:1003A0000148016070470000100C014001218140AC
:1003B0000148416170470000001001400121814067
:1003C000014801617047000000100140F0B53B4E4C
:1003D0003B4CB04203D1A66946F00406A661394EF3
:1003E000B04203D1A66946F00806A661364EB04277
:1003F00003D1A66946F01006A661344EB04203D17F
:10040000A66946F02006A661314EB04203D1A66926
:1004100046F04006A66100240F2900DD0124692A68
:1004200001D0492A02D1032B00D10124032B00DD86
:100430000124692A06D0492A04D06F2A02D04F2A03
:1004400000D00124692A01D0492A00D100256F2A51
:1004500001D04F2A00D1012503260222082915DAEE
:10046000076802EB810206FA02FC27EA0C07076024
:10047000076893401F430760026889008E40B243BB
:10048000026002688D402A43026015E0083947681F
:1004900002EB810206FA02FC27EA0C074760476874
:1004A00093401F434760426889008E40B2434260D8
:1004B00042688D402A4342602046F0BD000801405A
:1004C00000100240000C01400010014000140140E7
:1004D0000018014001490880704700003C040040BA
:1004E00070B53B4908883B4C82073B4DA4F1200680
:1004F000A4F1800018D50A8822F002020A8001784F
:10050000012901D1006A804728888107334802D435
:100510000088208003E000882188401A30802888E5
:1005200080F00200288070BD0A88520718D50A881A
:1005300022F004020A804178012901D1406A8047F3
:1005400028888106264802D40088608003E000885D
:100550006188401A7080288880F02000288070BD53
:100560000A88120718D50A8822F008020A808178C2
:10057000032901D1806A804728888105194802D45F
:100580000088A08003E00088A188401AB0802888F5
:1005900080F40070288070BD0A88D206FBD50A88D6
:1005A00022F010020A80C178012901D1C06A804777
:1005B000288881040C4802D40088E08003E0008889
:1005C000E188401AF080288880F40050288070BDAF
:1005D000102C014080000020202C0140342C0140D0
:1005E000382C01403C2C0140402C0140034801883C
:1005F00021F001010180024800690047102C0140F0
:100600000000002070B54FF08045288AC10740489F
:100610000AD0A989C90707D0298A21F001012982B6
:100620004069BDE870400047298A394C8A0738493B
:1006300004F18804A4F12006497916D52A8A22F00B
:1006400002022A82012901D1006B8047288C800791
:1006500002D4A88E208003E0A88E2188401A308022
:10066000288C80F00200288470BD2A8A520716D593
:100670002A8A22F004022A82012901D1406B804794
:10068000288C800602D4288F608003E0288F618840
:10069000401A7080288C80F02000288470BD298A40
:1006A000090717D5298A21F00801298281790129B2
:1006B00001D1806B8047288C800502D4A88FA08050
:1006C00003E0A88FA188401AB080288C80F40070C5
:1006D000288470BD298AC906FBD5298A21F010011A
:1006E0002982C179012901D1C06B8047288C8004FF
:1006F00003D4B5F84000E08004E0B5F84000E1889C
:10070000401AF080288C80F40050288470BD0000CE
:100710000000002070B543490888C20742480BD04A
:100720000A1F1288D20707D00A8822F001020A8025
:100730008069BDE8704000470A883B4C3B4D04F19E
:1007400090049207A4F1200618D50A8822F002022C
:100750000A80017A012901D1006C8047288881072D
:10076000334802D40088208003E000882188401AA2
:100770003080288880F00200288070BD0A885207E7
:1007800018D50A8822F004020A80417A012901D191
:10079000406C804728888106264802D40088608003
:1007A00003E000886188401A7080288880F020006B
:1007B000288070BD0A88120718D50A8822F008021E
:1007C0000A80817A012901D1806C804728888105BF
:1007D000194802D40088A08003E00088A188401A4C
:1007E000B080288880F40070288070BD0A88D20606
:1007F000FBD50A8822F010020A80C17A012901D1B2
:10080000C06C8047288881040C4802D40088E080AE
:1008100003E00088E188401AF080288880F40050C6
:10082000288070BD1004004000000020200400401B
:1008300034040040380400403C04004040040040C0
:1008400070B543490888C20742480BD00A1F128876
:10085000D20707D00A8822F001020A80C069BDE8E9
:10086000704000470A883B4C3B4D04F198049207C6
:10087000A4F1200618D50A8822F002020A80017B22
:10088000012901D1006D804728888107334802D4AF
:100890000088208003E000882188401A3080288862
:1008A00080F00200288070BD0A88520718D50A8897
:1008B00022F004020A80417B012901D1406D80476A
:1008C00028888106264802D40088608003E00088DA
:1008D0006188401A7080288880F02000288070BDD0
:1008E0000A88120718D50A8822F008020A80817B3C
:1008F000012901D1806D804728888105194802D4DB
:100900000088A08003E00088A188401AB080288871
:1009100080F40070288070BD0A88D206FBD50A8852
:1009200022F010020A80C17B012901D1C06D8047ED
:10093000288881040C4802D40088E08003E0008805
:10094000E188401AF080288880F40050288070BD2B
:10095000100800400000002020080040340800403B
:10096000380800403C0800404008004070B504468C
:100970000D46194919488C4203D1816941F400613F
:100980008161B4F1804F03D1C16941F00101C161BE
:1009900013498C4203D1C16941F00201C16111497F
:1009A0008C4203D1C16941F00401C161FFF78EFCA3
:1009B00006462046FFF78EFCB6FBF0F0B5FBF0F0E4
:1009C000010C4A1CB0FBF2F02185401EA085A084DA
:1009D0001120208070BD0000002C0140001002405A
:1009E000000400400008004002E008C8121F08C1CF
:1009F000002AFAD170477047002001E001C1121FA0
:100A0000002AFBD170470000FFF726FC084909487F
:100A1000FFF7ACFF084A02210648FFF7ABFB0023B3
:100A20006F2201210548FFF7D1FC00BFFEE700005F
:100A300000DD6D0000080040410A0008000C014084
:100A400000B50A4A11784FF00100012905D14FF095
:100A500000011160FFF7A2FC04E04FF001011160FA
:100A6000FFF794FC5DF804EB70470000A000002045
:100A7000900A000800000020A4000000E809000817
:100A8000340B0008A400002004040000F80900084A
:100A90000000000000000000000000000000000056
:100AA0000000000000000000000000000000000046
:100AB0000000000000000000000000000000000036
:100AC0000000000000000000000000000000000026
:100AD0000000000000000000000000000000000016
:100AE0000000000000000000000000000000000006
:100AF00000000000000000000000000000000000F6
:100B000000000000000000000000000000000000E5
:100B100000000000000000000000000000000000D5
:100B200000000000000000000000000000000000C5
:040B300000000000C1
:04000005080000ED02
:00000001FF
